
 Start         Length     Name                   Class
 0001:00000000 00002A6CH .text                   CODE
 0002:00000000 0000005CH .data                   DATA
 0002:0000005C 00000061H .bss                    BSS


Detailed map of segments

 0001:00000000 000000E6 C=CODE     S=.text    G=(none)   M=System   ACBP=A9
 0001:000000E8 000001EC C=CODE     S=.text    G=(none)   M=SysInit  ACBP=A9
 0001:000002D4 00000026 C=CODE     S=.text    G=(none)   M=DesignIntf ACBP=A9
 0001:000002FC 000000FE C=CODE     S=.text    G=(none)   M=Controls ACBP=A9
 0001:000003FC 0000000E C=CODE     S=.text    G=(none)   M=ActnList ACBP=A9
 0001:0000040C 0000000E C=CODE     S=.text    G=(none)   M=Contnrs  ACBP=A9
 0001:0000041C 0000003E C=CODE     S=.text    G=(none)   M=Classes  ACBP=A9
 0001:0000045C 0000000E C=CODE     S=.text    G=(none)   M=ActiveX  ACBP=A9
 0001:0000046C 00000038 C=CODE     S=.text    G=(none)   M=Messages ACBP=A9
 0001:000004A4 00000040 C=CODE     S=.text    G=(none)   M=Windows  ACBP=A9
 0001:000004E4 0000000E C=CODE     S=.text    G=(none)   M=Types    ACBP=A9
 0001:000004F4 0000000E C=CODE     S=.text    G=(none)   M=TypInfo  ACBP=A9
 0001:00000504 0000002E C=CODE     S=.text    G=(none)   M=SysUtils ACBP=A9
 0001:00000534 0000000E C=CODE     S=.text    G=(none)   M=SysConst ACBP=A9
 0001:00000544 0000000E C=CODE     S=.text    G=(none)   M=Variants ACBP=A9
 0001:00000554 0000000E C=CODE     S=.text    G=(none)   M=VarUtils ACBP=A9
 0001:00000564 0000000E C=CODE     S=.text    G=(none)   M=RTLConsts ACBP=A9
 0001:00000574 0000000E C=CODE     S=.text    G=(none)   M=Math     ACBP=A9
 0001:00000584 0000000E C=CODE     S=.text    G=(none)   M=ImgList  ACBP=A9
 0001:00000594 00000038 C=CODE     S=.text    G=(none)   M=CommCtrl ACBP=A9
 0001:000005CC 0000001E C=CODE     S=.text    G=(none)   M=Graphics ACBP=A9
 0001:000005EC 0000000E C=CODE     S=.text    G=(none)   M=Consts   ACBP=A9
 0001:000005FC 00000136 C=CODE     S=.text    G=(none)   M=Forms    ACBP=A9
 0001:00000734 0000000E C=CODE     S=.text    G=(none)   M=HelpIntfs ACBP=A9
 0001:00000744 0000000E C=CODE     S=.text    G=(none)   M=MultiMon ACBP=A9
 0001:00000754 00000038 C=CODE     S=.text    G=(none)   M=Imm      ACBP=A9
 0001:0000078C 0000000E C=CODE     S=.text    G=(none)   M=Menus    ACBP=A9
 0001:0000079C 0000000E C=CODE     S=.text    G=(none)   M=WinHelpViewer ACBP=A9
 0001:000007AC 0000000E C=CODE     S=.text    G=(none)   M=StdActns ACBP=A9
 0001:000007BC 00000016 C=CODE     S=.text    G=(none)   M=Dialogs  ACBP=A9
 0001:000007D4 00000038 C=CODE     S=.text    G=(none)   M=ShlObj   ACBP=A9
 0001:0000080C 00000038 C=CODE     S=.text    G=(none)   M=UrlMon   ACBP=A9
 0001:00000844 00000038 C=CODE     S=.text    G=(none)   M=WinInet  ACBP=A9
 0001:0000087C 00000038 C=CODE     S=.text    G=(none)   M=RegStr   ACBP=A9
 0001:000008B4 00000038 C=CODE     S=.text    G=(none)   M=ShellAPI ACBP=A9
 0001:000008EC 0000000E C=CODE     S=.text    G=(none)   M=Printers ACBP=A9
 0001:000008FC 00000038 C=CODE     S=.text    G=(none)   M=WinSpool ACBP=A9
 0001:00000934 00000016 C=CODE     S=.text    G=(none)   M=StdCtrls ACBP=A9
 0001:0000094C 00000038 C=CODE     S=.text    G=(none)   M=CommDlg  ACBP=A9
 0001:00000984 00000038 C=CODE     S=.text    G=(none)   M=Dlgs     ACBP=A9
 0001:000009BC 0000001E C=CODE     S=.text    G=(none)   M=ExtCtrls ACBP=A9
 0001:000009DC 0000000E C=CODE     S=.text    G=(none)   M=StrUtils ACBP=A9
 0001:000009EC 0000000E C=CODE     S=.text    G=(none)   M=Clipbrd  ACBP=A9
 0001:000009FC 0000000E C=CODE     S=.text    G=(none)   M=FlatSB   ACBP=A9
 0001:00000A0C 0000000E C=CODE     S=.text    G=(none)   M=DesignMenus ACBP=A9
 0001:00000A1C 0000000E C=CODE     S=.text    G=(none)   M=IniFiles ACBP=A9
 0001:00000A2C 000000D6 C=CODE     S=.text    G=(none)   M=DesignEditors ACBP=A9
 0001:00000B04 0000000E C=CODE     S=.text    G=(none)   M=Proxies  ACBP=A9
 0001:00000B14 0000000E C=CODE     S=.text    G=(none)   M=DesignConst ACBP=A9
 0001:00000B24 0000000E C=CODE     S=.text    G=(none)   M=Tabs     ACBP=A9
 0001:00000B34 0000002E C=CODE     S=.text    G=(none)   M=Grids    ACBP=A9
 0001:00000B64 0000000E C=CODE     S=.text    G=(none)   M=Mask     ACBP=A9
 0001:00000B74 0000000E C=CODE     S=.text    G=(none)   M=MaskUtils ACBP=A9
 0001:00000B84 0000000E C=CODE     S=.text    G=(none)   M=Buttons  ACBP=A9
 0001:00000B94 000003FC C=CODE     S=.text    G=(none)   M=PageInfo ACBP=A9
 0001:00000F90 00000070 C=CODE     S=.text    G=(none)   M=Win31Cst ACBP=A9
 0001:00001000 0000000E C=CODE     S=.text    G=(none)   M=LibHelp  ACBP=A9
 0001:00001010 00000974 C=CODE     S=.text    G=(none)   M=PageEdit ACBP=A9
 0001:00001984 000004EC C=CODE     S=.text    G=(none)   M=NoteBReg ACBP=A9
 0001:00001E70 00000016 C=CODE     S=.text    G=(none)   M=TabNotBk ACBP=A9
 0001:00001E88 0000000E C=CODE     S=.text    G=(none)   M=ComCtrls ACBP=A9
 0001:00001E98 0000000E C=CODE     S=.text    G=(none)   M=ListActns ACBP=A9
 0001:00001EA8 0000000E C=CODE     S=.text    G=(none)   M=ToolWin  ACBP=A9
 0001:00001EB8 00000038 C=CODE     S=.text    G=(none)   M=RichEdit ACBP=A9
 0001:00001EF0 0000000E C=CODE     S=.text    G=(none)   M=ExtActns ACBP=A9
 0001:00001F00 0000000E C=CODE     S=.text    G=(none)   M=Registry ACBP=A9
 0001:00001F10 0000000E C=CODE     S=.text    G=(none)   M=ExtDlgs  ACBP=A9
 0001:00001F20 0000000E C=CODE     S=.text    G=(none)   M=Mapi     ACBP=A9
 0001:00001F30 0000000E C=CODE     S=.text    G=(none)   M=ComStrs  ACBP=A9
 0001:00001F40 0000000E C=CODE     S=.text    G=(none)   M=Outline  ACBP=A9
 0001:00001F50 0000000E C=CODE     S=.text    G=(none)   M=FileCtrl ACBP=A9
 0001:00001F60 0000000E C=CODE     S=.text    G=(none)   M=FiltEdit ACBP=A9
 0001:00001F70 0000000E C=CODE     S=.text    G=(none)   M=DsnConst ACBP=A9
 0001:00001F80 00000864 C=CODE     S=.text    G=(none)   M=Win31Reg ACBP=A9
 0001:000027E4 00000285 C=CODE     S=.text    G=(none)   M=dcl31w   ACBP=A9
 0002:00000000 00000028 C=DATA     S=.data    G=DGROUP   M=SysInit  ACBP=A9
 0002:00000028 00000008 C=DATA     S=.data    G=DGROUP   M=NoteBReg ACBP=A9
 0002:00000030 00000008 C=DATA     S=.data    G=DGROUP   M=Win31Reg ACBP=A9
 0002:00001000 00000018 C=BSS      S=.bss     G=DGROUP   M=SysInit  ACBP=A9
 0002:00001018 00000004 C=BSS      S=.bss     G=DGROUP   M=Messages ACBP=A9
 0002:0000101C 00000004 C=BSS      S=.bss     G=DGROUP   M=Windows  ACBP=A9
 0002:00001020 00000004 C=BSS      S=.bss     G=DGROUP   M=CommCtrl ACBP=A9
 0002:00001024 00000004 C=BSS      S=.bss     G=DGROUP   M=Imm      ACBP=A9
 0002:00001028 00000004 C=BSS      S=.bss     G=DGROUP   M=ShlObj   ACBP=A9
 0002:0000102C 00000004 C=BSS      S=.bss     G=DGROUP   M=UrlMon   ACBP=A9
 0002:00001030 00000004 C=BSS      S=.bss     G=DGROUP   M=WinInet  ACBP=A9
 0002:00001034 00000004 C=BSS      S=.bss     G=DGROUP   M=RegStr   ACBP=A9
 0002:00001038 00000004 C=BSS      S=.bss     G=DGROUP   M=ShellAPI ACBP=A9
 0002:0000103C 00000004 C=BSS      S=.bss     G=DGROUP   M=WinSpool ACBP=A9
 0002:00001040 00000004 C=BSS      S=.bss     G=DGROUP   M=CommDlg  ACBP=A9
 0002:00001044 00000004 C=BSS      S=.bss     G=DGROUP   M=Dlgs     ACBP=A9
 0002:00001048 00000004 C=BSS      S=.bss     G=DGROUP   M=PageInfo ACBP=A9
 0002:0000104C 00000004 C=BSS      S=.bss     G=DGROUP   M=Win31Cst ACBP=A9
 0002:00001050 00000004 C=BSS      S=.bss     G=DGROUP   M=PageEdit ACBP=A9
 0002:00001054 00000004 C=BSS      S=.bss     G=DGROUP   M=NoteBReg ACBP=A9
 0002:00001058 00000004 C=BSS      S=.bss     G=DGROUP   M=RichEdit ACBP=A9
 0002:0000105C 00000004 C=BSS      S=.bss     G=DGROUP   M=Win31Reg ACBP=A9


  Address         Publics by Name

 0002:00001018       .1
 0002:00001020       .1
 0002:00001024       .1
 0002:00001028       .1
 0002:0000102C       .1
 0002:00001010       .1
 0002:00001058       .1
 0002:00001030       .1
 0002:00001034       .1
 0002:0000104C       .1
 0002:00001038       .1
 0002:00001044       .1
 0002:00001040       .1
 0002:00001050       .2
 0002:00001048       .2
 0002:0000103C       .3
 0002:0000101C       .3
 0002:00001054       .4
 0002:0000105C       .4
 0001:00002A44       @GetPackageInfoTable
 0001:00000220       @InitPkg
 0001:00002A4C       @PackageLoad
 0001:00000284       @PackageLoad
 0001:00002A58       @PackageUnload
 0001:00000290       @PackageUnload
 0001:00000120       AllocTlsBuffer
 0001:000005C4       CommCtrl
 0001:0000097C       CommDlg
 0001:00002A64       dcl31w
 0001:000009B4       Dlgs
 0001:000001CC       ExitProcessTLS
 0001:000001A4       ExitThreadTLS
 0001:000004A4       ExtTextOut
 0001:000004AC       Finalization
 0001:0000194C       Finalization
 0001:00002784       Finalization
 0001:00000594       Finalization
 0001:00001EB8       Finalization
 0001:00000754       Finalization
 0001:000008B4       Finalization
 0001:000007D4       Finalization
 0001:00000984       Finalization
 0001:0000080C       Finalization
 0001:0000094C       Finalization
 0001:0000087C       Finalization
 0001:00000844       Finalization
 0001:00001E10       Finalization
 0001:00000F58       Finalization
 0001:0000029C       Finalization
 0001:00000FC8       Finalization
 0001:0000046C       Finalization
 0001:000008FC       Finalization
 0001:000000E8       FreeLibrary
 0001:0000012C       GetTlsSize
 0002:0000100C       HInstance
 0001:00000784       Imm
 0001:000001F0       InitializeModule
 0001:00000178       InitProcessTLS
 0001:00000134       InitThreadTLS
 0001:000000F0       LocalAlloc
 0001:000000F8       LocalFree
 0001:0000049C       Messages
 0002:00000000       Module
 0002:00001000       ModuleIsLib
 0002:00001001       ModuleIsPackage
 0001:00001E5C       NoteBReg
 0001:0000197C       PageEdit
 0001:00000F88       PageInfo
 0001:00002428       Register
 0001:000008AC       RegStr
 0001:00001EE8       RichEdit
 0001:000008E4       ShellAPI
 0001:00000804       ShlObj
 0001:000002CC       SysInit
 0001:00000100       TlsAlloc
 0002:00001014       tlsBuffer
 0001:00000108       TlsFree
 0001:00000110       TlsGetValue
 0002:00001004       TlsIndex
 0002:AFFFC000       TlsLast
 0002:00000018       TlsProc
 0001:00000118       TlsSetValue
 0001:00001678       TNotebookEditDlg.AddClick
 0001:000017D8       TNotebookEditDlg.DeleteClick
 0001:0000151C       TNotebookEditDlg.EditClick
 0001:00001448       TNotebookEditDlg.FormCreate
 0001:000012DC       TNotebookEditDlg.GridDrawCell
 0001:0000191C       TNotebookEditDlg.HeaderSized
 0001:00001934       TNotebookEditDlg.HelpBtnClick
 0001:000014A0       TNotebookEditDlg.MoveClick
 0001:000012B8       TNotebookEditDlg.SetPageList
 0001:00001D5C       TNotebookEditor.ExecuteVerb
 0001:00001DF0       TNotebookEditor.GetVerb
 0001:00001E08       TNotebookEditor.GetVerbCount
 0001:00000F40       TPageInfoDlg.BitBtn3Click
 0001:00000E3C       TPageInfoDlg.GetPageContext
 0001:00000DC4       TPageInfoDlg.GetPageName
 0001:00000E90       TPageInfoDlg.OKClick
 0001:00000DDC       TPageInfoDlg.SetPageContext
 0001:00000DA8       TPageInfoDlg.SetPageName
 0001:00001CDC       TPageListProperty.Edit
 0001:00001C8C       TPageListProperty.GetAttributes
 0001:00001C98       TPageListProperty.GetValue
 0001:00001BBC       TPageNameProperty.GetAttributes
 0001:00001C70       TPageNameProperty.GetValue
 0001:00001BC8       TPageNameProperty.GetValues
 0001:00001C84       TPageNameProperty.SetValue
 0001:00002374       TTabbedNotebookEditor.ExecuteVerb
 0001:00002408       TTabbedNotebookEditor.GetVerb
 0001:00002420       TTabbedNotebookEditor.GetVerbCount
 0001:000022F4       TTabPageListProperty.Edit
 0001:000022A4       TTabPageListProperty.GetAttributes
 0001:000022B0       TTabPageListProperty.GetValue
 0001:000021D4       TTabPageNameProperty.GetAttributes
 0001:00002288       TTabPageNameProperty.GetValue
 0001:000021E0       TTabPageNameProperty.GetValues
 0001:0000229C       TTabPageNameProperty.SetValue
 0001:000001FC       UninitializeModule
 0001:0000083C       UrlMon
 0002:00000028       Verbs
 0002:00000030       Verbs
 0001:00000FF8       Win31Cst
 0001:000027D0       Win31Reg
 0001:000004DC       Windows
 0001:00000874       WinInet
 0001:0000092C       WinSpool


  Address         Publics by Value

 0002:AFFFC000       TlsLast
 0001:000000E8       FreeLibrary
 0001:000000F0       LocalAlloc
 0001:000000F8       LocalFree
 0001:00000100       TlsAlloc
 0001:00000108       TlsFree
 0001:00000110       TlsGetValue
 0001:00000118       TlsSetValue
 0001:00000120       AllocTlsBuffer
 0001:0000012C       GetTlsSize
 0001:00000134       InitThreadTLS
 0001:00000178       InitProcessTLS
 0001:000001A4       ExitThreadTLS
 0001:000001CC       ExitProcessTLS
 0001:000001F0       InitializeModule
 0001:000001FC       UninitializeModule
 0001:00000220       @InitPkg
 0001:00000284       @PackageLoad
 0001:00000290       @PackageUnload
 0001:0000029C       Finalization
 0001:000002CC       SysInit
 0001:0000046C       Finalization
 0001:0000049C       Messages
 0001:000004A4       ExtTextOut
 0001:000004AC       Finalization
 0001:000004DC       Windows
 0001:00000594       Finalization
 0001:000005C4       CommCtrl
 0001:00000754       Finalization
 0001:00000784       Imm
 0001:000007D4       Finalization
 0001:00000804       ShlObj
 0001:0000080C       Finalization
 0001:0000083C       UrlMon
 0001:00000844       Finalization
 0001:00000874       WinInet
 0001:0000087C       Finalization
 0001:000008AC       RegStr
 0001:000008B4       Finalization
 0001:000008E4       ShellAPI
 0001:000008FC       Finalization
 0001:0000092C       WinSpool
 0001:0000094C       Finalization
 0001:0000097C       CommDlg
 0001:00000984       Finalization
 0001:000009B4       Dlgs
 0001:00000DA8       TPageInfoDlg.SetPageName
 0001:00000DC4       TPageInfoDlg.GetPageName
 0001:00000DDC       TPageInfoDlg.SetPageContext
 0001:00000E3C       TPageInfoDlg.GetPageContext
 0001:00000E90       TPageInfoDlg.OKClick
 0001:00000F40       TPageInfoDlg.BitBtn3Click
 0001:00000F58       Finalization
 0001:00000F88       PageInfo
 0001:00000FC8       Finalization
 0001:00000FF8       Win31Cst
 0001:000012B8       TNotebookEditDlg.SetPageList
 0001:000012DC       TNotebookEditDlg.GridDrawCell
 0001:00001448       TNotebookEditDlg.FormCreate
 0001:000014A0       TNotebookEditDlg.MoveClick
 0001:0000151C       TNotebookEditDlg.EditClick
 0001:00001678       TNotebookEditDlg.AddClick
 0001:000017D8       TNotebookEditDlg.DeleteClick
 0001:0000191C       TNotebookEditDlg.HeaderSized
 0001:00001934       TNotebookEditDlg.HelpBtnClick
 0001:0000194C       Finalization
 0001:0000197C       PageEdit
 0001:00001BBC       TPageNameProperty.GetAttributes
 0001:00001BC8       TPageNameProperty.GetValues
 0001:00001C70       TPageNameProperty.GetValue
 0001:00001C84       TPageNameProperty.SetValue
 0001:00001C8C       TPageListProperty.GetAttributes
 0001:00001C98       TPageListProperty.GetValue
 0001:00001CDC       TPageListProperty.Edit
 0001:00001D5C       TNotebookEditor.ExecuteVerb
 0001:00001DF0       TNotebookEditor.GetVerb
 0001:00001E08       TNotebookEditor.GetVerbCount
 0001:00001E10       Finalization
 0001:00001E5C       NoteBReg
 0001:00001EB8       Finalization
 0001:00001EE8       RichEdit
 0001:000021D4       TTabPageNameProperty.GetAttributes
 0001:000021E0       TTabPageNameProperty.GetValues
 0001:00002288       TTabPageNameProperty.GetValue
 0001:0000229C       TTabPageNameProperty.SetValue
 0001:000022A4       TTabPageListProperty.GetAttributes
 0001:000022B0       TTabPageListProperty.GetValue
 0001:000022F4       TTabPageListProperty.Edit
 0001:00002374       TTabbedNotebookEditor.ExecuteVerb
 0001:00002408       TTabbedNotebookEditor.GetVerb
 0001:00002420       TTabbedNotebookEditor.GetVerbCount
 0001:00002428       Register
 0001:00002784       Finalization
 0001:000027D0       Win31Reg
 0001:00002A44       @GetPackageInfoTable
 0001:00002A4C       @PackageLoad
 0001:00002A58       @PackageUnload
 0001:00002A64       dcl31w
 0002:00000000       Module
 0002:00000018       TlsProc
 0002:00000028       Verbs
 0002:00000030       Verbs
 0002:00001000       ModuleIsLib
 0002:00001001       ModuleIsPackage
 0002:00001004       TlsIndex
 0002:0000100C       HInstance
 0002:00001010       .1
 0002:00001014       tlsBuffer
 0002:00001018       .1
 0002:0000101C       .3
 0002:00001020       .1
 0002:00001024       .1
 0002:00001028       .1
 0002:0000102C       .1
 0002:00001030       .1
 0002:00001034       .1
 0002:00001038       .1
 0002:0000103C       .3
 0002:00001040       .1
 0002:00001044       .1
 0002:00001048       .2
 0002:0000104C       .1
 0002:00001050       .2
 0002:00001054       .4
 0002:00001058       .1
 0002:0000105C       .4


Bound resource files

PageInfo.dfm
PageEdit.dfm
dcl31w.res
win31reg.dcr
C:\TEMP\dtf29C6.tmp


Program entry point at 0001:00002A64
